 imx_xvc

 Timestamp is 4da293ba (Mon Apr 11 17:38:02 2011)

 Preferred load address is 10000000

 Start         Length     Name                   Class
 0001:00000000 00000004H .CRT$XCA                CODE
 0001:00000004 00000004H .CRT$XCZ                CODE
 0001:00000008 00000004H .CRT$XIA                CODE
 0001:0000000c 00000004H .CRT$XIZ                CODE
 0001:00000010 00000004H .CRT$XPA                CODE
 0001:00000014 00000004H .CRT$XPZ                CODE
 0001:00000018 00000004H .CRT$XTA                CODE
 0001:0000001c 00000004H .CRT$XTZ                CODE
 0001:00000020 00000140H .rdata                  CODE
 0001:00000160 00000024H .rdata$debug            CODE
 0001:00000184 00001fd4H .text                   CODE
 0001:00002158 00000004H .xdata                  CODE
 0001:0000215c 0000003cH .idata$2                CODE
 0001:00002198 00000014H .idata$3                CODE
 0001:000021ac 000000b8H .idata$4                CODE
 0001:00002264 00000068H .idata$6                CODE
 0001:000022d0 00000104H .edata                  CODE
 0002:00000000 000000b8H .idata$5                DATA
 0002:000000b8 00000008H .data                   DATA
 0002:000000c0 0000001cH .bss                    DATA
 0003:00000000 00000170H .pdata                  DATA

  Address         Publics by Value              Rva+Base       Lib:Object

 0000:00000000       ___safe_se_handler_count   00000000     <absolute>
 0000:00000000       ___safe_se_handler_table   00000000     <absolute>
 0001:00000000       __xc_a                     10001000     corelib0:crt0init.obj
 0001:00000004       __xc_z                     10001004     corelib0:crt0init.obj
 0001:00000008       __xi_a                     10001008     corelib0:crt0init.obj
 0001:0000000c       __xi_z                     1000100c     corelib0:crt0init.obj
 0001:00000010       __xp_a                     10001010     corelib0:crt0init.obj
 0001:00000014       __xp_z                     10001014     corelib0:crt0init.obj
 0001:00000018       __xt_a                     10001018     corelib0:crt0init.obj
 0001:0000001c       __xt_z                     1000101c     corelib0:crt0init.obj
 0001:0000003c       ??_C@_1CC@BJPGGDNC@?$AAU?$AAS?$AAB?$AA_?$AAC?$AAL?$AAO?$AAC?$AAK?$AA_?$AAG?$AAA?$AAT?$AAI?$AAN?$AAG?$AA?$AA@ 1000103c     i_usbclock.obj
 0001:00000060       ??_C@_1BC@GDFGLIEL@?$AAO?$AAT?$AAG?$AAG?$AAr?$AAo?$AAu?$AAp?$AA?$AA@ 10001060     usb_xvc_mx25_topaz_v1:i_xvc.obj
 0001:00000074       ??_C@_1BG@HHFAGDDC@?$AAO?$AAT?$AAG?$AAS?$AAu?$AAp?$AAp?$AAo?$AAr?$AAt?$AA?$AA@ 10001074     usb_xvc_mx25_topaz_v1:i_xvc.obj
 0001:0000008c       ??_C@_17DJGGJCGD@?$AAI?$AAr?$AAq?$AA?$AA@ 1000108c     usb_xvc_mx25_topaz_v1:i_xvc.obj
 0001:00000094       ??_C@_1O@LBBNFMDB@?$AAM?$AAe?$AAm?$AAL?$AAe?$AAn?$AA?$AA@ 10001094     usb_xvc_mx25_topaz_v1:i_xvc.obj
 0001:000000a4       ??_C@_1BA@INLDIDEN@?$AAM?$AAe?$AAm?$AAB?$AAa?$AAs?$AAe?$AA?$AA@ 100010a4     usb_xvc_mx25_topaz_v1:i_xvc.obj
 0001:00000130       ??_C@_1BA@EKAPLICF@?$AAU?$AAS?$AAB?$AAF?$AAu?$AAn?$AAc?$AA?$AA@ 10001130     usb_xvc_mx25_topaz_v1:i_xvc.obj
 0001:00000140       ??_C@_1BA@JAHEEJIA@?$AAU?$AAS?$AAB?$AAX?$AAC?$AAV?$AAR?$AA?$AA@ 10001140     usb_xvc_mx25_topaz_v1:i_xvc.obj
 0001:00000150       ??_C@_1BA@MLDLNLBG@?$AAU?$AAS?$AAB?$AAH?$AAo?$AAs?$AAt?$AA?$AA@ 10001150     usb_xvc_mx25_topaz_v1:i_xvc.obj
 0001:00000184       BSPGetUSBControllerType    10001184 f   hwinit.obj
 0001:00000434       InitializeOTGTransceiver   10001434 f   hwinit.obj
 0001:00000618       RegisterCallback           10001618 f   hwinit.obj
 0001:00000638       BSPUsbResetPHY             10001638 f   hwinit.obj
 0001:00000654       BSPUsbSetPHYEnable         10001654 f   hwinit.obj
 0001:00000670       USBClockGatingLock         10001670 f   i_usbclock.obj
 0001:000006ac       BSPUSBClockCreateFileMapping 100016ac f   i_usbclock.obj
 0001:0000074c       BSPUSBClockSwitch          1000174c f   i_usbclock.obj
 0001:00000840       USBClockInit               10001840 f   i_usbclock.obj
 0001:00000848       PowerDownSchemeExist       10001848 f   i_usbutils.obj
 0001:000008a4       BSPUsbEnableLowPowerIntr   100018a4 f   i_usbutils.obj
 0001:000008f8       BSPUsbSetBusConfig         100018f8 f   i_usbutils.obj
 0001:00000908       BSPUSBInterruptControl     10001908 f   i_usbutils.obj
 0001:0000094c       FslUfnIsUSBKitlEnable      1000194c f   usb_xvc_mx25_topaz_v1:i_xvc.obj
 0001:000009b8       DllEntry                   100019b8 f   usb_xvc_mx25_topaz_v1:i_xvc.obj
 0001:00000afc       XVC_ISTMain                10001afc f   usb_xvc_mx25_topaz_v1:i_xvc.obj
 0001:00001064       XVC_Deinit                 10002064 f   usb_xvc_mx25_topaz_v1:i_xvc.obj
 0001:000010ec       XVC_Open                   100020ec f   usb_xvc_mx25_topaz_v1:i_xvc.obj
 0001:000010f0       XVC_Close                  100020f0 f   usb_xvc_mx25_topaz_v1:i_xvc.obj
 0001:000010f8       XVC_PowerDown              100020f8 f   usb_xvc_mx25_topaz_v1:i_xvc.obj
 0001:000010fc       XVC_PowerUp                100020fc f   usb_xvc_mx25_topaz_v1:i_xvc.obj
 0001:000011ac       XVC_Read                   100021ac f   usb_xvc_mx25_topaz_v1:i_xvc.obj
 0001:000011b4       XVC_Write                  100021b4 f   usb_xvc_mx25_topaz_v1:i_xvc.obj
 0001:000011bc       XVC_Seek                   100021bc f   usb_xvc_mx25_topaz_v1:i_xvc.obj
 0001:000011c4       XVC_IOControl              100021c4 f   usb_xvc_mx25_topaz_v1:i_xvc.obj
 0001:0000141c       XVC_Init                   1000241c f   usb_xvc_mx25_topaz_v1:i_xvc.obj
 0001:00001a68       GetDeviceRegistryParams    10002a68 f   usb_xvc_mx25_topaz_v1:i_registry.obj
 0001:00001c04       Sleep                      10002c04 f   coredll:COREDLL.dll
 0001:00001c14       KernelIoControl            10002c14 f   coredll:COREDLL.dll
 0001:00001c24       InterlockedCompareExchange 10002c24 f   coredll:COREDLL.dll
 0001:00001c34       GetLastError               10002c34 f   coredll:COREDLL.dll
 0001:00001c44       MapViewOfFile              10002c44 f   coredll:COREDLL.dll
 0001:00001c54       CreateFileMappingW         10002c54 f   coredll:COREDLL.dll
 0001:00001c64       CloseHandle                10002c64 f   coredll:COREDLL.dll
 0001:00001c74       EventModify                10002c74 f   coredll:COREDLL.dll
 0001:00001c84       DisableThreadLibraryCalls  10002c84 f   coredll:COREDLL.dll
 0001:00001c94       ExitThread                 10002c94 f   coredll:COREDLL.dll
 0001:00001ca4       InterruptDone              10002ca4 f   coredll:COREDLL.dll
 0001:00001cb4       InterruptInitialize        10002cb4 f   coredll:COREDLL.dll
 0001:00001cc4       InterruptDisable           10002cc4 f   coredll:COREDLL.dll
 0001:00001cd4       LeaveCriticalSection       10002cd4 f   coredll:COREDLL.dll
 0001:00001ce4       EnterCriticalSection       10002ce4 f   coredll:COREDLL.dll
 0001:00001cf4       WaitForSingleObject        10002cf4 f   coredll:COREDLL.dll
 0001:00001d04       SetInterruptEvent          10002d04 f   coredll:COREDLL.dll
 0001:00001d14       CreateEventW               10002d14 f   coredll:COREDLL.dll
 0001:00001d24       StringCchCatW              10002d24 f   coredll:COREDLL.dll
 0001:00001d34       StringCchCopyW             10002d34 f   coredll:COREDLL.dll
 0001:00001d44       LocalFree                  10002d44 f   coredll:COREDLL.dll
 0001:00001d54       CeSetThreadPriority        10002d54 f   coredll:COREDLL.dll
 0001:00001d64       CreateThread               10002d64 f   coredll:COREDLL.dll
 0001:00001d74       InitializeCriticalSection  10002d74 f   coredll:COREDLL.dll
 0001:00001d84       LocalAlloc                 10002d84 f   coredll:COREDLL.dll
 0001:00001d94       SetThreadPriority          10002d94 f   coredll:COREDLL.dll
 0001:00001da4       RegQueryValueExW           10002da4 f   coredll:COREDLL.dll
 0001:00001db4       RegCloseKey                10002db4 f   coredll:COREDLL.dll
 0001:00001dc4       RegOpenKeyExW              10002dc4 f   coredll:COREDLL.dll
 0001:00001dd4       OpenDeviceKey              10002dd4 f   coredll:COREDLL.dll
 0001:00001de4       MmUnmapIoSpace             10002de4 f   ceddk:CEDDK.dll
 0001:00001df4       MmMapIoSpace               10002df4 f   ceddk:CEDDK.dll
 0001:00001e04       DDKClockSetGatingMode      10002e04 f   cspddk:CSPDDK.dll
 0001:00001e14       DDKClockGetGatingMode      10002e14 f   cspddk:CSPDDK.dll
 0001:00001e24       DDKClockConfigBaud         10002e24 f   cspddk:CSPDDK.dll
 0001:00001e34       _DllEntryCRTStartup        10002e34 f   corelib0:pegdentry.obj
 0001:00001e78       __GSHandlerCheckCommon     10002e78 f   corelib0:gshandler.obj
 0001:00001eb0       __GSHandlerCheck           10002eb0 f   corelib0:gshandler.obj
 0001:00001ed0       __security_init_cookie     10002ed0 f   corelib0:seccinit.obj
 0001:00001f1c       __security_check_cookie    10002f1c f   corelib0:armsecgs.obj
 0001:00001f2c       __gsfailure                10002f2c     corelib0:armsecgs.obj
 0001:00002030       _cexit                     10003030 f   corelib0:cexit.obj
 0001:00002040       _initterm                  10003040 f   corelib0:crt0dat.obj
 0001:0000206c       _cinit                     1000306c f   corelib0:crt0dat.obj
 0001:000020cc       __crt_ExitProcess          100030cc f   corelib0:exitproc_proxy.obj
 0001:000020d8       memset                     100030d8 f   corelib1:COREDLL.dll
 0001:000020e8       memcpy                     100030e8 f   corelib1:COREDLL.dll
 0001:000020f8       wcslen                     100030f8 f   corelib1:COREDLL.dll
 0001:00002108       wcstoul                    10003108 f   corelib1:COREDLL.dll
 0001:00002118       __security_gen_cookie2     10003118 f   corelib1:COREDLL.dll
 0001:00002128       __report_gsfailure         10003128 f   corelib1:COREDLL.dll
 0001:00002138       free                       10003138 f   corelib1:COREDLL.dll
 0001:00002148       TerminateProcess           10003148 f   coredll:COREDLL.dll
 0001:0000215c       __IMPORT_DESCRIPTOR_COREDLL 1000315c     coredll:COREDLL.dll
 0001:00002170       __IMPORT_DESCRIPTOR_CEDDK  10003170     ceddk:CEDDK.dll
 0001:00002184       __IMPORT_DESCRIPTOR_CSPDDK 10003184     cspddk:CSPDDK.dll
 0001:00002198       __NULL_IMPORT_DESCRIPTOR   10003198     coredll:COREDLL.dll
 0002:00000000       __imp_MmUnmapIoSpace       10004000     ceddk:CEDDK.dll
 0002:00000004       __imp_MmMapIoSpace         10004004     ceddk:CEDDK.dll
 0002:00000008       \177CEDDK_NULL_THUNK_DATA  10004008     ceddk:CEDDK.dll
 0002:0000000c       __imp_GetLastError         1000400c     coredll:COREDLL.dll
 0002:00000010       __imp_MapViewOfFile        10004010     coredll:COREDLL.dll
 0002:00000014       __imp_CreateFileMappingW   10004014     coredll:COREDLL.dll
 0002:00000018       __imp_CloseHandle          10004018     coredll:COREDLL.dll
 0002:0000001c       __imp_EventModify          1000401c     coredll:COREDLL.dll
 0002:00000020       __imp_DisableThreadLibraryCalls 10004020     coredll:COREDLL.dll
 0002:00000024       __imp_ExitThread           10004024     coredll:COREDLL.dll
 0002:00000028       __imp_InterruptDone        10004028     coredll:COREDLL.dll
 0002:0000002c       __imp_InterruptInitialize  1000402c     coredll:COREDLL.dll
 0002:00000030       __imp_InterruptDisable     10004030     coredll:COREDLL.dll
 0002:00000034       __imp_LeaveCriticalSection 10004034     coredll:COREDLL.dll
 0002:00000038       __imp_EnterCriticalSection 10004038     coredll:COREDLL.dll
 0002:0000003c       __imp_WaitForSingleObject  1000403c     coredll:COREDLL.dll
 0002:00000040       __imp_InterlockedCompareExchange 10004040     coredll:COREDLL.dll
 0002:00000044       __imp_CreateEventW         10004044     coredll:COREDLL.dll
 0002:00000048       __imp_StringCchCatW        10004048     coredll:COREDLL.dll
 0002:0000004c       __imp_StringCchCopyW       1000404c     coredll:COREDLL.dll
 0002:00000050       __imp_LocalFree            10004050     coredll:COREDLL.dll
 0002:00000054       __imp_CeSetThreadPriority  10004054     coredll:COREDLL.dll
 0002:00000058       __imp_CreateThread         10004058     coredll:COREDLL.dll
 0002:0000005c       __imp_InitializeCriticalSection 1000405c     coredll:COREDLL.dll
 0002:00000060       __imp_LocalAlloc           10004060     coredll:COREDLL.dll
 0002:00000064       __imp_SetThreadPriority    10004064     coredll:COREDLL.dll
 0002:00000068       __imp_RegQueryValueExW     10004068     coredll:COREDLL.dll
 0002:0000006c       __imp_RegCloseKey          1000406c     coredll:COREDLL.dll
 0002:00000070       __imp_RegOpenKeyExW        10004070     coredll:COREDLL.dll
 0002:00000074       __imp_OpenDeviceKey        10004074     coredll:COREDLL.dll
 0002:00000078       __imp_KernelIoControl      10004078     coredll:COREDLL.dll
 0002:0000007c       __imp_SetInterruptEvent    1000407c     coredll:COREDLL.dll
 0002:00000080       __imp_Sleep                10004080     coredll:COREDLL.dll
 0002:00000084       __imp_free                 10004084     corelib1:COREDLL.dll
 0002:00000088       __imp_memset               10004088     corelib1:COREDLL.dll
 0002:0000008c       __imp_memcpy               1000408c     corelib1:COREDLL.dll
 0002:00000090       __imp_wcslen               10004090     corelib1:COREDLL.dll
 0002:00000094       __imp_wcstoul              10004094     corelib1:COREDLL.dll
 0002:00000098       __imp___security_gen_cookie2 10004098     corelib1:COREDLL.dll
 0002:0000009c       __imp___report_gsfailure   1000409c     corelib1:COREDLL.dll
 0002:000000a0       __imp_TerminateProcess     100040a0     coredll:COREDLL.dll
 0002:000000a4       \177COREDLL_NULL_THUNK_DATA 100040a4     coredll:COREDLL.dll
 0002:000000a8       __imp_DDKClockGetGatingMode 100040a8     cspddk:CSPDDK.dll
 0002:000000ac       __imp_DDKClockSetGatingMode 100040ac     cspddk:CSPDDK.dll
 0002:000000b0       __imp_DDKClockConfigBaud   100040b0     cspddk:CSPDDK.dll
 0002:000000b4       \177CSPDDK_NULL_THUNK_DATA 100040b4     cspddk:CSPDDK.dll
 0002:000000b8       __security_cookie          100040b8     corelib0:seccinit.obj
 0002:000000bc       __security_cookie_complement 100040bc     corelib0:seccinit.obj
 0002:000000c0       m_hUSBClockGatingHandle    100040c0     i_usbclock.obj
 0002:000000c4       pUSBClkGating              100040c4     i_usbclock.obj
 0002:000000c8       g_pXVC                     100040c8     usb_xvc_mx25_topaz_v1:i_xvc.obj
 0002:000000cc       gfsvaim                    100040cc     usb_xvc_mx25_topaz_v1:i_xvc.obj
 0002:000000d0       _exitflag                  100040d0     corelib0:cexit.obj
 0002:000000d4       __onexitend                100040d4     <common>
 0002:000000d8       __onexitbegin              100040d8     <common>

 entry point at        0001:00001e34

 Static symbols

 0001:0000018c       ConfigOTGHost              1000118c f   hwinit.obj
 0001:000002c4       ConfigOTGClient            100012c4 f   hwinit.obj
 0001:000005c8       BSPUsbXvrSetPhyPowerMode   100015c8 f   hwinit.obj
 0001:000009cc       USBControllerRun           100019cc f   usb_xvc_mx25_topaz_v1:i_xvc.obj
 0001:00000a6c       USBControllerReset         10001a6c f   usb_xvc_mx25_topaz_v1:i_xvc.obj
 0001:00001100       PowerDown                  10002100 f   usb_xvc_mx25_topaz_v1:i_xvc.obj
 0001:0000165c       GetStringParam             1000265c f   usb_xvc_mx25_topaz_v1:i_registry.obj
 0001:000017ac       GetMultiDWordParam         100027ac f   usb_xvc_mx25_topaz_v1:i_registry.obj
 0001:00001970       GetBinParam                10002970 f   usb_xvc_mx25_topaz_v1:i_registry.obj
 0001:00001f70       doexit                     10002f70 f   corelib0:cexit.obj
